:100000000C944A000C9469000C9469000C946900EB
:100010000C9469000C9469000C9469000C946900BC
:100020000C9469000C9469000C9469000C946900AC
:100030000C9469000C9469000C9469000C9469009C
:100040000C9469000C9469000C9469000C9469008C
:100050000C9469000C9469000C9469000C9469007C
:100060000C9469000C9469000C9469000C9469006C
:100070000C9469000C9469000C9469000C9469005C
:100080000C9469000C9469000C9469000C9469004C
:100090000C94690011241FBECFEFD0E1DEBFCDBFAD
:1000A00011E0A0E0B1E0E0EAF1E000E00BBF02C047
:1000B00007900D92A030B107D9F711E0A0E0B1E0B0
:1000C00001C01D92A030B107E1F70E94A6000C9478
:1000D000CF000C940000CF93DF93CDB7DEB7E2E200
:1000E000F0E01082E1E2F0E01082E5E2F0E0108260
:1000F000E4E2F0E01082E8E2F0E01082E7E2F0E013
:100100001082EBE2F0E01082EAE2F0E01082EEE230
:10011000F0E01082EDE2F0E080E18083E1E3F0E0E6
:100120001082E0E3F0E01082DF91CF910895CF9349
:10013000DF93CDB7DEB7E0E6F0E088E18083E0E66C
:10014000F0E087E08083DF91CF910895CF93DF9334
:10015000CDB7DEB724970FB6F894DEBF0FBECDBF84
:100160000E9497000E946B0000C0A895ECE2F0E0AE
:100170008081992780729070009749F4AEE2B0E0D8
:10018000EEE2F0E090818FEE89238C93EECFAEE229
:10019000B0E0EEE2F0E0808180618C93E6CFFFCFAB
:00000001FF
